:03000000020240B9
:0C024000787FE4F6D8FD7581070200030A
:10020E0012022E7590FFC290C295C296AF03AE0237
:10021E0012022E7590FFC290C295C296AF03AE0227
:10022E00E4FDFCC3ED9FEC9E50070DBD00010C805C
:02023E00F222AA
:100003007590FF7B967A00C290C293C292C295C24A
:1000130094C2971202287590FFC29012022875901D
:10002300FFC2901202287590FFC293C29712022A50
:100033007590FFC292C295C29412022A7590FF1264
:10004300022A12022EC290C293C292C295C294C2D5
:1000530097C29612020E7590FFC290C295C296AFD8
:1000630003AE0212020E7590FF12022A12022EC272
:1000730090C293C292C295C294C29712022E7590F7
:10008300FF1202287590FFC292C295C294C29712C2
:10009300022A7590FF1202287590FFC290C293C284
:1000A30092C295C294C29712022A7590FF12022A35
:1000B30012022EC292C29512022E7590FFC293C2F3
:1000C3009412022A7590FFC293C29712022A759066
:1000D300FFC2921202287590FFC293C29712022A9E
:1000E3007590FFC293C29412022A7590FFC292C206
:1000F3009512022A7590FF12022A12022EC2901242
:10010300022E7590FFC29012022A7590FFC290C210
:1001130093C292C295C294C2971202287590FFC2ED
:100123009012022A7590FFC29012022A7590FF1254
:10013300022A12022EC292C295C294C297C296128A
:10014300022E7590FFC293C29512022A7590FFC2C8
:1001530090C29512022A7590FFC293C29512022A89
:100163007590FFC292C295C294C2971202287590ED
:10017300FF12022A12022EC290C293C292C295C2E9
:1001830094C297C29612022E7590FFC290C2951226
:10019300022A7590FFC290C29512022A7590FFC27F
:1001A30090C295C29412022A7590FFC293C292C262
:1001B300971202287590FF12022A12022EC290C2D1
:1001C30093C292C295C294C297C29612022E7590A0
:1001D300FFC29212022A7590FFC29512022A7590ED
:1001E300FFC29412022A7590FFC290C293C292C2B8
:1001F30095C294C2971202287590FF12022A120226
:0B0203002E7F887E1312022E02000ADC
:00000001FF
